S02B00002F686F6D652F766F6F72627572672F446576656C6F706D656E742F4F70656E424C542F5461726765E0
S31508000000008000200D1C00085D1C00085D1C00080F
S3150800001000000000000000000000000000000000D2
S315080000200000000000000000000000005D1C000841
S3150800003000000000000000005D1C00085D1C0008B0
S315080000405D1C00085D1C00085D1C00085D1C00089E
S315080000505D1C00085D1C00085D1C00085D1C00088E
S315080000605D1C00085D1C00085D1C00085D1C00087E
S315080000705D1C00085D1C00085D1C00085D1C00086E
S315080000805D1C00085D1C00085D1C00085D1C00085E
S315080000905D1C00085D1C00085D1C00085D1C00084E
S315080000A05D1C00085D1C00085D1C00085D1C00083E
S311080000B05D1C00085D1C00085D1C0008B3
S315080000BC10B5064C2378002B07D1054B002B02D024
S315080000CC044800E000BF0123237010BDD4000020B3
S315080000DC00000000A81C0008044B10B5002B03D028
S315080000EC0349044800E000BF10BDC04600000000EC
S315080000FCD8000020A81C0008002243088B4274D3A1
S3150800010C03098B425FD3030A8B4244D3030B8B42FE
S3150800011C28D3030C8B420DD3FF22090212BA030C07
S3150800012C8B4202D31212090265D0030B8B4219D3E8
S3150800013C00E0090AC30B8B4201D3CB03C01A524108
S3150800014C830B8B4201D38B03C01A5241430B8B4250
S3150800015C01D34B03C01A5241030B8B4201D30B0339
S3150800016CC01A5241C30A8B4201D3CB02C01A524160
S3150800017C830A8B4201D38B02C01A5241430A8B4223
S3150800018C01D34B02C01A5241030A8B4201D30B020C
S3150800019CC01A5241CDD2C3098B4201D3CB01C01A26
S315080001AC524183098B4201D38B01C01A5241430930
S315080001BC8B4201D34B01C01A524103098B4201D31E
S315080001CC0B01C01A5241C3088B4201D3CB00C01A8B
S315080001DC524183088B4201D38B00C01A5241430803
S315080001EC8B4201D34B00C01A5241411A00D2014628
S315080001FC524110467047FFE701B5002000F006F89B
S3150800020C02BDC0460029F7D076E770477047C0464E
S3150800021C72B6704762B67047F0B5D6464F4680B58B
S3150800022C8DB081468A46019202A801F037FA049BE2
S3150800023C0093002501E00135EDB2112D1FD8134BA3
S3150800024C6A00D65C9B185F78F41901344B465C43FC
S3150800025C21000098FFF7D6FF0029ECD12100009861
S3150800026CFFF74AFF80B253461880013880B2084B14
S3150800027C9842E0D8019B1E705F70012000E00020B8
S3150800028C0DB00CBC91469A46F0BDC046EC1C000855
S3150800029CFF03000070B588B06B46991C01230B80D0
S315080002AC1E4B1B886A4613801D48FFF7B5FF0128AD
S315080002BC03D093211B4800F0EBFB1B4E300000F0DB
S315080002CCE6FE05AD280000F0F5FF0024AC71EC71D4
S315080002DC2C726C72AC72EC72AC70EC706B461B7850
S315080002EC013B2B716B465B78013B6B716B4602339A
S315080002FC1B882B802900300000F0D6FE01A88472DA
S3150800030CC47201230373048044808480C4800481EE
S3150800031C437300F04DFF08B070BDC046C01C000802
S3150800032C20A10700C41C00080064004010B586B064
S3150800033C01AB00221A720F4C01945A72997200235F
S3150800034C05E0C45C01AAD218D4720133DBB28B4225
S3150800035CF7D301A9084800F0BDFF040001E000F03E
S3150800036C55FC2100044801F01BF80228F7D006B00A
S3150800037C10BDC046E10700000064004030B587B0E8
S3150800038C04000021144801F089F8002802D1002045
S3150800039C07B030BD01AD2A0000210F4801F030F836
S315080003AC2B7A002B05D10D4B019A9A4206D00020C8
S315080003BC00E000200128EBD1002307E00120F9E733
S315080003CC01AAD218D27AE2540133DBB201AA927A84
S315080003DC9342F5D3DCE7C04600640040670600008C
S315080003EC10B5FFF715FF10BD70B508E0461C4D1C7F
S315080003FC0B78037000F00AFC300029002200541E0A
S3150800040CA4B2002AF2D170BD10B500F03BFA002850
S3150800041C00D110BD00F0ECFD0028FAD000F0AEFBC0
S3150800042C00F042FA0121012001F040FA00F02EFA00
S3150800043C0100C02280208005FFF7D6FF032001F0BB
S3150800044C5FFA00F023FA4468FFF7E4FEA047E0E7FA
S3150800045C70B50500002401E00134E4B2122C15D85D
S3150800046C00F0D4FB63001B199A00094BD358AB4216
S3150800047CF2D8620012199000054A121852689B1895
S3150800048C9D42E9D2024B1B18187A00E0FF2070BD7A
S3150800049C101D000870B505000024122C10D800F0A9
S315080004ACB5FB63001B199A00074B9B181B7AAB42CA
S315080004BC02D00134E4B2F0E71300034A985801E07D
S315080004CC0120404270BDC046101D000870B50500DD
S315080004DC0024122C10D800F099FB63001B199A0003
S315080004EC064B9B181B7AAB4202D00134E4B2F0E7F8
S315080004FC024B9B18586800E0002070BD101D0008C0
S3150800050C10B5CB0509D10368994208D002C08022E0
S3150800051C9200FFF769FF012000E0002010BD0120C2
S3150800052CFCE7F8B507000068FFF792FFFF282AD00A
S3150800053C00F0C2FF342000F0D7FF00F0DBFF0128E3
S3150800054C14D000257F2D15D8AB003A68D418FB18A3
S3150800055C5E6800F05BFB3100200001F00FF8042800
S3150800056C0AD123689E420CD10135EBE700F0B4FFA3
S3150800057C002404E0012400E0002400F0ADFF200074
S3150800058CF8BD0024F9E70024F9E7000070B504006B
S3150800059C0D000C4B984208D00B4B994207D0FFF72D
S315080005ACC0FF002804D1002408E0084C00E0054CE4
S315080005BC29002000FFF7A4FF002801D0200070BDF9
S315080005CC0024FBE7F402002000200008F0000020BD
S315080005DCF0B5C64600B507000C0015001E004B0A00
S315080005EC5B029846036801330DD03B68984505D0E5
S315080005FC41463800FFF7CAFF071E26D03B68E41AA7
S3150800060C3C1904340CE04146FFF77AFF0028ECD17C
S3150800061C18E02B78237001340135013E002E10D0DA
S3150800062C00F0F4FA3B1DE31A0A4A9342F1D98021E9
S3150800063C890041443800FFF7A9FF071E07D0041D9F
S3150800064CE7E7012004BC9046F0BD0020FAE700203D
S3150800065CF8E7C046FF01000070B504000D0088429B
S3150800066C39D8032839D9162901D9002034E000F0E5
S3150800067C23FF342000F038FF00F03CFF01281ED081
S3150800068C2000FFF707FF06002800FFF703FF04000A
S3150800069C2800FFF71BFF2518013DAD1B0135ED0A98
S315080006ACADB20024AC4212D200F0B0FAE002301817
S315080006BC00F046FF042806D10134A4B2F2E700F094
S315080006CC0BFF002008E000F007FF002004E000F014
S315080006DC03FF012000E0002070BD0020FCE70000AD
S315080006EC01235B42024A1360024A13607047C046F4
S315080006FCF0000020F402002070B504000D0016006E
S3150800070CFFF7A6FEFF2818D060190138FFF7A0FEE0
S3150800071CFF2814D0630A5B020A4A934206D02B00C0
S3150800072C320021000848FFF753FF70BD2B0032003A
S3150800073C21000648FFF74CFFF7E70020F5E70020F5
S3150800074CF3E7C04600200008F0000020F402002061
S3150800075CF8B504000F00FFF77BFE0500E019013819
S3150800076CFFF776FEFF2D06D0FF2806D001002800DD
S3150800077CFFF772FFF8BD0020FCE70020FAE700003F
S3150800078C00B583B0104B1B6801331BD00E4A536857
S3150800079C91688C466344D1688C46634411698C46CF
S315080007AC634451698C46634491698C466344D269A7
S315080007BC9B185B42019301AA04210448FFF79CFF8E
S315080007CC03B000BD0120FBE7F4020020C02000089E
S315080007DC0E4B1B680E4A12689B180E4A12689B1819
S315080007EC0D4A12689B180D4A12689B180C4A126817
S315080007FC9B180C4A12689B180B4A12689B18002BFC
S3150800080C01D0002070470120FCE7C04600200008F4
S3150800081C04200008082000080C20000810200008F6
S3150800082C1420000818200008C020000810B50B4B2F
S3150800083C1B68013304D00948FFF773FE002809D05A
S3150800084C074B1B68013306D00548FFF76AFE0028DC
S3150800085C00D0012010BD0120FCE7C046F4020020A0
S3150800086CF0000020004870470020000810B5FFF77C
S3150800087C37FF10BD10B5FFF73FFF10BD10B5FFF7DA
S3150800088C67FF10BD10B5FFF7A3FF10BD10B5FFF736
S3150800089CE9FF10BD10B5FFF773FF002800D110BD96
S315080008ACFFF7C4FFFBE700000022014B1A607047F4
S315080008BC10E000E010B5FFF7F7FF054B054A5A6044
S315080008CC00229A6005211960034B1A6010BDC046B8
S315080008DC10E000E07FBB0000F8040020044B1B6806
S315080008ECDB0303D5034A1368013313607047C0460C
S315080008FC10E000E0F804002010B5FFF7EFFF014BFD
S3150800090C186810BDF804002010B5040080210948A9
S3150800091C01F08AF8002801D1002010BDA1B20548C3
S3150800092C01F070F88021034801F07EF80028F9D010
S3150800093C0120F2E70044004010B5040020210648C7
S3150800094C01F072F8012801D0002010BD024801F010
S3150800095C5DF820700120F8E70044004010B586B019
S3150800096CE1231B020093002301930293039305933F
S3150800097C0C330493074C6946200000F0CBFF80210A
S3150800098C4901200001F046F80121200001F02EF85B
S3150800099C06B010BD0044004070B506000D00402995
S315080009AC0AD82800FFF7B0FF012803D083210E4888
S315080009BC00F06EF8002406E07F210B4800F068F87A
S315080009CCEFE70134A4B2ABB29C420BD200F01EF98D
S315080009DC305DFFF799FF0128F3D08C21024800F00F
S315080009EC57F8EEE770BDC046F41D000870B5050053
S315080009FC234B1C78002C15D12248FFF79DFF0128A4
S31508000A0C01D0200070BD1F4B1B78002BF9D0FFF7C7
S31508000A1C73FF1D4B186000221C4B1A700132184BC1
S31508000A2C1A70EEE7194B1B7801331648C018FFF7F6
S31508000A3C83FF040001280BD0FFF75EFF124B1B68DF
S31508000A4C6433984219D900220D4B1A700024D8E742
S31508000A5C0E4B1A780132D2B21A700A4B1B789A428C
S31508000A6C01D00024CDE792B2064901312800FFF7E0
S31508000A7CBBFC0022024B1A70C3E70024C1E7C04630
S31508000A8C3D050020FC040020400500203E05002002
S31508000A9C10B500F0BBF8FCE710B500F0AFF801286C
S31508000AAC03D0094B1B78012B00D010BDFFF724FF90
S31508000ABC064B1B68F533FF339842F6D30022024BDC
S31508000ACC1A70FFF7A1FCF0E7440500204805002042
S31508000ADC10B50122044B1A70FFF70EFF034B186072
S31508000AECFFF7DAFF10BDC046440500204805002074
S31508000AFC10B5FFF775FC00F085F8FFF7DBFEFFF77E
S31508000B0CB5FE00F00DF8FFF7E3FF10BD10B500F0C9
S31508000B1C7DF8FFF7E3FE00F013F8FFF7BDFF10BDF5
S31508000B2C10B500F0E9F9FFF7B5FB044C0123237067
S31508000B3CFFF714FF0023237010BDC046C000002029
S31508000B4C10B50C48FFF71AFC012805D00948FFF721
S31508000B5C4DFF012807D010BD0122074B1A70054816
S31508000B6C00F0EAF9F2E70022034B1A70014800F08C
S31508000B7CE3F9F0E74C050020C000002070470000A0
S31508000B8C70B505000C000A4B1B78012B06D0084BD8
S31508000B9C1B78002B06D000F0C7F970BDC9B2FFF759
S31508000BACC5FBF4E7E1B22800FFF7F6FEF3E7C0460B
S31508000BBCC0000020074B1B78022B05D0032B05D051
S31508000BCC012B05D0402070470020FCE70020FAE7EF
S31508000BDC0820F8E7C0000020074B1B78022B05D02D
S31508000BEC032B05D0012B05D0402070470020FCE7CD
S31508000BFC0020FAE70820F8E7C000002010B500F03E
S31508000C0C89F910BD10B500F001FA10BD10B500F049
S31508000C1C02FA10BD10B5002304E001785B18DBB2AC
S31508000C2C013021004C1E0029F7D11360012010BD9C
S31508000C3C0022014B5A7070478C050020034BFE228C
S31508000C4CDA7018710221BA3A995270478C0500204D
S31508000C5C10B5054C00232370FFF7EAFFFF23E3705A
S31508000C6C0122BB3BE25210BD8C050020064BFF222D
S31508000C7CDA7000221A71597859719A71DA711A72E6
S31508000C8C06214432995270478C05002010B5002075
S31508000C9CFFF7D4FF10BD0000094BFF22DA70094A92
S31508000CAC9A6400221A715A719A710721D971002116
S31508000CBC1972597299720831442299527047C04672
S31508000CCC8C050020F81E0008044BFF22DA704268D7
S31508000CDC9A640121442299527047C0468C0500201B
S31508000CEC10B5084CFF23E370E21D4168A06CFFF7B2
S31508000CFC91FF207100236371A37108224433E252D9
S31508000D0C10BDC0468C05002010B53120FFF796FFA4
S31508000D1C10BD000070B5084CFF23E3700025257143
S31508000D2C6571FFF747FFA071E57125726572072299
S31508000D3C4423E25270BDC0468C05002070B5FFF7FF
S31508000D4C77FF0D4C01252570FF23E370EF3B2371CC
S31508000D5C00236371FFF72EFFA071FFF73DFFE071CB
S31508000D6CFFF73AFF000A20726572A572082244231F
S31508000D7CE252FFF77BFD70BD8C05002070B50500AF
S31508000D8C4478FFF717FF0138844211DC0A4C6A785D
S31508000D9C201DA16CFFF728FBFF23E3706B78A26C70
S31508000DAC94466344A3646B7801334422A35270BD02
S31508000DBC2220FFF743FFFAE78C05002070B50400E4
S31508000DCC4578FFF7F7FE0138854212DC61680B4D52
S31508000DDCA9646278281DFFF707FBFF23EB7063787D
S31508000DECAA6C94466344AB64637801334422AB52D1
S31508000DFC70BD2220FFF722FFFAE7C0468C050020BB
S31508000E0C70B504000E4B9D6CFFF7D4FE411E621C98
S31508000E1C2800FFF72FFD00280DD0094CFF23E3709F
S31508000E2CFFF7C8FE0138A36C9C466044A0640122F7
S31508000E3C4423E25270BD3130FFF700FFFAE7C04693
S31508000E4C8C05002070B504004578FFF7B3FE023810
S31508000E5C854210DC134BFF22DA700121BB3A9952FA
S31508000E6C617800290BD1FFF715FD002814D1313014
S31508000E7CFFF7E4FE10E02220FFF7E0FE0CE0094B3A
S31508000E8C986CA21CFFF7F6FC002806D06378054A76
S31508000E9C916C8C466344936470BD3130FFF7CEFE7B
S31508000EACFAE7C0468C05002010B5094B9B6C4168C7
S31508000EBC1800FFF7E3FC002806D0054BFF22DA7072
S31508000ECC0121BB3A995210BD3130FFF7B7FEFAE74C
S31508000EDC8C05002010B5FFF797FA034BFF22DA7042
S31508000EEC0121BB3A995210BD8C05002010B589B268
S31508000EFCFFF746FE10BD0000054B00221A709A64D7
S31508000F0C43215A5401315A529A705A707047C04646
S31508000F1C8C050020034B1B78002B01D00120704751
S31508000F2C0020FCE78C05002000214323014AD154FC
S31508000F3C7047C0468C05002010B50378FF2B04D0EB
S31508000F4C294A1278012A14D010BDFFF7F7FE43235D
S31508000F5C254AD35C012B42D04423234AD15E00296F
S31508000F6CF2DD100001224323C2540330FFF7BEFF03
S31508000F7CEAE73733DAB2352A2DD893001B4AD35809
S31508000F8C9F46FFF7FBFEE2E7FFF718FFDFE7FFF7E1
S31508000F9C9BFEDCE7FFF7A4FED9E7FFF77DFED6E755
S31508000FACFFF774FED3E7FFF761FED0E7FFF750FEB5
S31508000FBCCDE7FFF725FFCAE7FFF744FFC7E7FFF7BB
S31508000FCCA9FEC4E7FFF770FFC1E7FFF783FFBEE78B
S31508000FDCFFF79AFEBBE72020FFF730FEB7E7102095
S31508000FECFFF72CFEB8E7C0468C050020201E00082B
S31508000FFC10B500F045F880218901034800F032FB52
S3150800100C002800D0012010BD0008004810B5642047
S3150800101C00F006F810BD10B500F008F810BD000079
S3150800102C014B18807047C046D805002010B5FFF74D
S3150800103C63FC104B1B68984212D30F4B1B78002B82
S3150800104C0FD101220C4B1A7020219020C00500F0FC
S3150800105C10FBFFF751FC094B1B881818054B186039
S3150800106C10BD0022044B1A7020219020C00500F0F8
S3150800107C02FBEEE7DC050020DA050020D805002087
S3150800108C10B520219020C00500F0F5FA10BD10B55A
S3150800109C8024A4040121200000F024FC0021200057
S315080010AC00F020FC10BD0000036802229343036085
S315080010BC0368013A13430360002300E001334268D6
S315080010CCD20702D4394A9342F8D14368DB076AD56A
S315080010DC8B79012B3BD00368802293430360CB7931
S315080010EC012B39D003684022934303600B7A012BFA
S315080010FC37D003682022934303604B7A012B35D0F3
S3150800110C03681022934303608B7A012B33D0036850
S3150800111C082293430360CB7A012B31D0036804224F
S3150800112C934303608B789B07CA78120613430A7994
S3150800113C120413434A79120513430A88013A1343D6
S3150800114CC361036801229343036000231EE003680E
S3150800115C802213430360C2E70368402213430360EB
S3150800116CC4E70368202213430360C6E7036810220A
S3150800117C13430360C8E70368082213430360CAE7EE
S3150800118C0368042213430360CCE701334268D20791
S3150800119C02D5064A9342F8D14368DB0701D40120ED
S315080011AC02E0002000E000207047C046FFFFFF0069
S315080011BC70B5837A01252A009A403D4B8024A400F9
S315080011CC1959294319518725AD005959D44321403A
S315080011DC5951037B002B18D1354D832189006B5847
S315080011EC23406B50837AC1880904468831434833B7
S315080011FCDB005951837A81880904058829434833C9
S3150800120CDB002B4DAC4663445960037B012B1FD086
S3150800121CC37A002B36D1264D812189006B58234081
S3150800122C6B500389002B05D1214D852189006B58FC
S3150800123C1C406C500389012B2BD0437B012B2FD0E0
S3150800124C1B49802292008B58012083438B5070BD1A
S3150800125C174D832189006B5813436B50837A018889
S3150800126C0904468831434833DB005951837A81880F
S3150800127C0904C58829434833DB000D4DAC46634445
S3150800128C5960C5E70A4D812189006B5813436B5089
S3150800129CC7E7074C85218900635813436350CCE78D
S315080012AC034987239B00C8580243CA50C8E7C0465F
S315080012BC0064004000238371C37103724372837206
S315080012CCC3728370C37003330371013B4371013BD3
S315080012DC03807047F0B503008268520107D4826810
S315080012EC12014CD48268D2004BD5022000E00020B3
S315080012FC042843D00200040018342401E6580125BA
S3150800130C3540E5500E7A002E3DD12500E6580C687E
S3150800131C64054F7A3C433443EC508D7A0F242C40A9
S3150800132C8C72150018352D015C1966680F27BE439B
S3150800133C666066688F7A3E4366608C7B24064E7BB5
S3150800134C360434430E7B36023443CE7A34431201C8
S3150800135C9A1816008936FF3634608C7C24064E7C27
S3150800136C360434430E7C36023443C97B21438D3212
S3150800137CFF321160EA5801210A43EA50F0BD0120F8
S3150800138CB6E70420B4E7050018352D01EF584C686C
S3150800139CE40034434E7A34433C43EC50BDE700003A
S315080013AC012914D0002903D0022914D0002302E005
S315080013BC8368104A13400F4A934214D00FD90E4A29
S315080013CC934212D00D4A934211D1012010E0836842
S315080013DC094A1340EFE78368084A1340EBE7002BEA
S315080013EC05D1022004E0012002E0012000E00020E3
S315080013FCC0B2704703000004000300080000031085
S3150800140C30B50B001B331B011C58042323401372E5
S3150800141C38D10B001B331B011B585B0D13600B00DB
S3150800142C1B331B011D5802242C405472C3185D68CB
S3150800143C0F242C4094725B681B0AD3740B01C318D7
S3150800144C1C00B934FF342568D57225682D0A157326
S3150800145C25682D0C55732468240E9473BD33FF33FD
S3150800146C1C68D4731C68240A14741C68240C5474E1
S3150800147C1B681B0E937400290BD003692022134397
S3150800148C036130BD0B001B331B011B58DB08536073
S3150800149CC5E7C36820221343C360F2E7002903D0CB
S315080014AC012905D0002002E0C068032318407047C4
S315080014BC006903231840FAE7044B1B691B0604D57D
S315080014CC024B034A5A60034A5A607047002002408E
S315080014DC23016745AB89EFCD024A136980210B437B
S315080014EC1361704700200240014BD8607047C04614
S315080014FC00200240094BDB68DB070BD4074BDB6883
S3150800150CDB0601D502207047044BDB685B0703D565
S3150800151C0320F8E70120F6E70420F4E70020024050
S3150800152C10B50400FFF7E6FF02E0FFF7E3FF013C06
S3150800153C012801D1002CF8D1002C00D1052010BDB2
S3150800154C70B50500B0200003FFF7EAFF042800D0A9
S3150800155C70BD094C236902263343236165612369EF
S3150800156C402213432361B0200003FFF7D9FF2369F8
S3150800157CB3432361ECE7C0460020024030B583B084
S3150800158C05000C0000230193B0200003FFF7C8FFE9
S3150800159C042801D003B030BD104A136901210B434E
S315080015AC1361A3B22B80B0200003FFF7B9FF042800
S315080015BC05D00A4A136901218B431361EAE7023500
S315080015CC0195019B240C1C80B0200003FFF7A8FF93
S315080015DC024A136901218B431361DBE700200240A1
S315080015EC70B500222FE0836855000324AC40A34352
S315080015FC836083684C79AC402343836083881504E5
S3150800160C2D0C0124AC40A343838086888C79AC408E
S3150800161CA3B2334383800468550003231E00AE40EF
S3150800162CB443046004680E79AE4034430460C4685D
S3150800163C1604F60BB3409C43C460C368CC79AC4023
S3150800164C2343C36001320F2A0BD8012393400C683D
S3150800165C1C40A342F6D10B79013BDBB2012BDAD83D
S3150800166CC1E770BD038A0B4201D1002070470120E7
S3150800167CFCE7816170470185704730B507230B403D
S3150800168C9B009A40C908083189000C580F259D40C3
S3150800169CAC430C500B581A430A5030BDF8B504002D
S315080016AC744B58680C23184004284DD007D90828C1
S315080016BC4ED00C2865D1704B2360002003E000281F
S315080016CC5FD16E4B23606B4A516809090F230B4097
S315080016DC6B4FFB5CDBB226683100D9400B006160AE
S315080016EC55682D0A07212940795CC9B2CB40A360FD
S315080016FC126BD20549D4634AE2605E4A126B5206F3
S3150800170C4DD4614A22615B4A126BD2064BD45B4AB2
S3150800171C6261584A126B920747D1A361554A116BFD
S3150800172CC022920211425BD1E361524A116BC0226C
S3150800173C1203114200D076E023624E4B1B6B1B063C
S3150800174C00D493E06062F8BD4C4B23600020BAE7E6
S3150800175C484B5D685A68C0235B02AD0C0F200540E8
S3150800176C02351A4203D1494868432060ABE7414B1E
S3150800177CDB6A0F21194001314048FEF7BDFC68436E
S3150800178CF3E73E4B236000209DE73A4A5268520421
S3150800179C02D45A08E260B0E79A08E260ADE7802204
S315080017AC12022261AFE76661B3E7324A116B032274
S315080017BC0A40012A0ED02F4A116B03220A40022A2C
S315080017CC0AD02C4A116B03220A40032AA6D12B4AAB
S315080017DCA261A3E7A661A1E780221202A2619DE796
S315080017EC244A126BC02189020A40802149028A4286
S315080017FC13D0204A126BC02189020A408021890223
S3150800180C8A420CD01B4A126BC02189020A408A42B2
S3150800181C00D08AE7194AE26187E7E66185E7802204
S3150800182C1202E26181E7134B1B6BC02212031340B1
S3150800183C8022D202934213D00E4B1B6BC02212038A
S3150800184C13408022120393420CD00A4B1B6BC02206
S3150800185C12031340934200D06FE7084B23626CE7E0
S3150800186C26626AE780231B02236266E7024B6362E1
S3150800187C69E7C04600100240006CDC0200127A00D0
S3150800188CC4000020809FD5001280000000093D008E
S3150800189C002904D1044A5369834353617047024AA9
S315080018AC536918435061F9E700100240002904D126
S315080018BC044A9369834393617047024A93691843B0
S315080018CC9061F9E700100240002904D1044AD36953
S315080018DC8343D3617047024AD3691843D061F9E749
S315080018EC00100240002904D1044A1369834313618A
S315080018FC7047024A136918431061F9E70010024051
S3150800190C034A136803218B43184310607047C0467B
S3150800191C00000140F0B58DB004000D0003680122EB
S3150800192C9343036043682A4A13408A681343436007
S3150800193C0368284A13404A68C9680A4329690A434E
S3150800194C134303608368244A13406A69134383600C
S3150800195C02A8FFF7A3FE214B9C4227D0204B9C42A2
S3150800196C26D0204B9C4225D0049E23681B0423D5E5
S3150800197C76002B68019319003000FEF7BDFB0700B3
S3150800198C01993000FEF73EFC2B685B08994200D3A0
S3150800199C013723681B0405D57B0807221A40124B0E
S315080019AC1F401743BBB2A3810DB0F0BD089EDCE700
S315080019BC099EDAE70A9ED8E72B68019319003000CE
S315080019CCFEF79AFB070001993000FEF71BFCDBE7D4
S315080019DCFFCFFFFFF3E9FFFFFFFCFFFF00380140D5
S315080019EC0044004000480040F0FF0000002904D1E4
S315080019FC036801229343036070470368012213436B
S31508001A0C0360F9E7C905C90D01857047808CC005C7
S31508001A1CC00D70478368034A134083608368194373
S31508001A2C81607047FFEFFFFFC369194201D100209F
S31508001A3C70470120FCE700001122144B1A60144B66
S31508001A4C5A685A605A685A605A6812490A405A6063
S31508001A5C5968A02292030A435A60196880225204D4
S31508001A6C0A431A600A4B1B689B01FBD5084B5A683C
S31508001A7C03218A435A605A6801390A435A60044B4F
S31508001A8C5A680C231340082BF9D1704700200240E2
S31508001A9C00100240FF7FC0FF10B5124B1A680121D7
S31508001AAC0A431A605A68104802405A601A680F4866
S31508001ABC02401A601A680E4802401A605A680D48A5
S31508001ACC02405A60DA6A0F208243DA621A6B0A48B5
S31508001ADC02401A635A6B8A435A6300229A60FFF7CC
S31508001AECABFF10BD001002400CB8FFF8FFFFF6FE66
S31508001AFCFFFFFBFFFFFFC0FFACFEFFFFF0B5C646BE
S31508001B0C00B582B08027BF0201213800FFF7C0FE5E
S31508001B1C2023009301266B461E7100249C71032317
S31508001B2C98466B4642465A71DC719025ED05694616
S31508001B3C2800FFF755FD20212800FFF79CFD012101
S31508001B4C80200003FFF7A4FE6B461C71DC71802312
S31508001B5C9B01009369462448FFF742FD0121380092
S31508001B6CFFF7B2FE01213800FFF792FE012202218F
S31508001B7C2800FFF782FD012203212800FFF77DFDCF
S31508001B8C0C2300936B4642465A7102271F719C71AF
S31508001B9CDE7169462800FFF723FD012180208004A9
S31508001BACFFF792FE01218020C002FFF771FE0F4D50
S31508001BBC042208212800FFF760FD042209212800C9
S31508001BCCFFF75BFDC0239B0000936B461F714246D3
S31508001BDC5A719C71DE7169462800FFF701FD02B047
S31508001BEC04BC9046F0BDC0460008004800040048F6
S31508001BFC10B5FFF783FFFEF77BFFFEF787FFFCE7C1
S31508001C0C0D488546002103E00C4B5B5843500431C4
S31508001C1C0B480C4B42189A42F6D30B4A02E00023A7
S31508001C2C13600432094B9A42F9D3FFF735FF00F0DB
S31508001C3C11F8FFF7DDFFFEE700800020081F0008FB
S31508001C4CC0000020D4000020D4000020E0050020AD
S31508001C5CFEE7000070B500260C4D0D4C641BA41055
S31508001C6CA64209D1002600F019F80A4D0A4C641B45
S31508001C7CA410A64205D170BDB300EB58984701369F
S31508001C8CEEE7B300EB5898470136F2E7001F000859
S31508001C9C001F0008001F0008041F0008F8B5C046FE
S31508001CACF8BC08BC9E467047F8B5C046F8BC08BCDC
S30908001CBC9E4670477B
S31508001CC0010100002E2E2F2E2E2F2E2E2F2E2E2FD8
S31508001CD0536F757263652F41524D434D305F5354B0
S31508001CE04D333246302F63616E2E630005020602BD
S31508001CF0060307030803090309040A040B040C0472
S31508001D000C050D050E050F050F0610061007100821
S31508001D100020000800080000040000000028000851
S31508001D200008000005000000003000080008000058
S31508001D300600000000380008000800000700000040
S31508001D4000400008000800000800000000480008DD
S31508001D500008000009000000005000080008000004
S31508001D600A00000000580008000800000B000000E8
S31508001D7000600008000800000C0000000068000869
S31508001D80000800000D0000000070000800080000B0
S31508001D900E00000000780008000800000F00000090
S31508001DA00080000800800000100000000000010804
S31508001DB0008000001100000000800108008000007B
S31508001DC01200000000000208008000001300000056
S31508001DD000800208008000001400000000000308CC
S31508001DE00080000015000000008003080080000045
S31508001DF0160000002E2E2F2E2E2F2E2E2F2E2E2F93
S31508001E00536F757263652F41524D434D305F53547E
S31508001E104D333246302F756172742E630000000010
S31508001E20BE0F0008E20F0008E20F0008DC0F0008EA
S31508001E30E20F0008E20F0008D60F0008C40F0008DA
S31508001E40D00F0008CA0F0008E20F0008E20F0008CA
S31508001E50E20F0008E20F0008E20F0008E20F000890
S31508001E60E20F0008E20F0008E20F0008E20F000880
S31508001E70E20F0008E20F0008E20F0008E20F000870
S31508001E80E20F0008E20F0008E20F0008E20F000860
S31508001E90E20F0008E20F0008E20F0008E20F000850
S31508001EA0E20F0008E20F0008E20F0008E20F000840
S31508001EB0E20F0008E20F0008E20F0008E20F000830
S31508001EC0E20F0008E20F0008A00F0008940F0008B0
S31508001ED08E0F00089A0F0008E20F0008E20F0008AC
S31508001EE0E20F0008A60F0008E20F0008AC0F000872
S31508001EF0B20F0008B80F00084F70656E424C5400C8
S30908001F00E5000008E2
S30908001F04BD00000806
S31508001F0804000000000000000102030401020304A3
S30908001F180607080999
S70508001C0DC9
